:060000008A110A123428E7
:10000800FF00030E83120313D700D70E0A08D80087
:100018000408D9008A110A120B1D2D285D088100D9
:100028002030DE073F300318013EFF3A013EDD0075
:100038000B11FF30E91B2328E807031CE907EB1B1A
:100048002828EA07031CEB07ED1B2D28EC07031CE7
:10005800ED077C08DA007D08DB007E08DC00C22999
:100068008B138312031385018601FF3083168500E5
:10007800FF3086008B1306308312A000A101A20175
:100088008730831681004E308312DD00DE01810047
:10009800A0308B00DF01FF30E201E301E800E90056
:1000A800E401E501EA00EB00E601E701EC00ED0000
:1000B8008128E10003105F0D623E8400831360080D
:1000C8008000840A61088000692883120313DF0A0C
:1000D8005F08033A0319DF0103105F0D8313623EC3
:1000E80084000008840A000403196928801B692811
:1000F80000088A0084030008820007309F00C701B7
:10010800C801831605100130840084076230840713
:100118008313CF308000840A0230800083125F0886
:10012800013A031D98286928023084008407623048
:100138008407831353308000840A063080005F08E8
:10014800023A031DA8286928CD0103110319AD2817
:10015800AE28BE294D08003A0319B328C228B83082
:10016800E00000305D286928831203132108220665
:100178008A110A12031DC128B728E928E1010130B4
:10018800E0005F0884008407683084078313840ACA
:100198008017840360088000840A61088000D830D2
:1001A800E00000305D286928831203132108220625
:1001B8008A110A12031DE9285F0884008407683041
:1001C80084078313840A801FD72803110319ED2895
:1001D800EE2875292208D500210855060319F528A7
:1001E800FE28CF010130FF3ACF09013E0319CF0A9B
:1001F800CE001629D201233055070318D20A8313DB
:100208005218831784000008D600D50A2008550222
:1002180003180F291029D5015508A200CF01560847
:10022800CE0016290310CF1F0314031C1C291D29F7
:1002380075294E08D00050087F39013A031925293D
:10024800462950088039003A03192B294429480ABD
:100258000339C80004304802031C33293F29D2015E
:100268003B3048070318D20A8313521883178400B7
:100278000008C7004129C70141298430CD04452918
:100288004D11742950087F39063A03194C295E2903
:1002980050088039003A031952295C294708013A65
:1002A800031D57295B290130C7028130CD045D2920
:1002B8004D10742950087F39073A031964297429A5
:1002C80050088039003A03196A2973294708FF3A08
:1002D800031D6F297229C70A8230CD047429CD10F5
:1002E800E9284D088039003A031D7B29A429CD133C
:1002F800E1010E30E0005F0884008407683084075D
:100308008313840A8017840360088000840A6108C4
:1003180080009230E00001305D28692883120313C1
:10032800210822068A110A12031DA3295F088400E6
:100338008407683084078313840A801F9129BD29A4
:100348004D080139003A031DAA29B1294708013A85
:10035800031DAF29B1290130C7024D080239003AFF
:10036800031DB729BD294708FF3A031DBC29BD292C
:10037800C70AA9284B088A004A0882004908083990
:10038800003A0319C829CA290514CB290510C90A36
:1003980036088604E101FA30E0000000E00BD129BC
:1003A8000000E1013F08E000E0080319E02900002F
:1003B8000000E00BDC29000043088605E101400845
:1003C800E000E0080319ED2900000000E00BE9292E
:1003D800000044088605E1014108E000E00803192F
:1003E800FA2900000000E00BF62900004508860500
:1003F800E1014208E000E0080319072A00000000B4
:10040800E00B032A0000460886055C08FE005B082E
:10041800FD005A08FC005908840058088A0057084B
:100428008300FF0E7F0E09008312AA01AB01831619
:1004380022088312AC00AD01AE0183162308831293
:10044800AF0083162208850423088604043083122B
:10045800A900831621088A00200882000130AD0017
:10046800AE0108302E02031C3A2A782A2A082D05E4
:10047800003A031D402A742A2E082C07AF002B08C7
:100488002D05003A031D492A4A2AAF17831221086D
:10049800013EF500200875020318532A542AF50175
:1004A800220875060319592A5F2A01308316B000FD
:1004B800B009B00A742A8316B10183122108233EB9
:1004C80083160318B10A831383163118831784001F
:1004D8002F08800075088312A1008316B001742AC2
:1004E8000310AD0DAE0A352A29088A0028088200B3
:1004F80083122C08003A031D822AA52A0508B30096
:100508000508B2000508B3040508B2050508B304D8
:100518000508B2052B08B1000508AB0031082B0609
:10052800B0002B08B3042B08B20533083206B1001B
:10053800310830042C05003A031DA32AA52A0330EC
:10054800A9002908003A031DAA2ACA2AFF30A907C8
:100558002908003A0319B12ACA2A2A082B062C05A9
:10056800B0003008003A031DBA2ACA2A2B082C0505
:10057800AA0030088316AA0083122A088316AB0043
:10058800AC010230A900CA30A800322A831621081B
:100598008A0020088200C23083160313A200A30138
:1005A8000230A100DB30A0008A110A12182A0311B8
:1005B8000319DF2AE02A0A2B02308316A100E6304D
:1005C800A0007C2A8312E001E1015F08840084070F
:1005D800683084078313840A8017840360088000C6
:1005E800840A61088000FC30E00002305D28692838
:1005F800831203135F088400840768308407831319
:10060800840A8A110A12801FFB2ADB2A74088A00CE
:1006180073088200DD01DC0102305C028A110A12D3
:10062800031C172B5B2BDF015C08DE000310DE0DBB
:10063800DF0D5E08873E0318DF0ADE000730DF079C
:100648005E08DE002B2B5F088A005E0882002723E5
:1006580083160313DA00DB0103118A110A12031946
:10066800362B372B412B5A085902031C3C2B3D2BA8
:10067800412B5A08D902DB0A302BDD08031D4A2B0F
:100688005B08003A0319492B4A2B592B0130DD002E
:100698005B08303EDE008313581883175708840020
:1006A8005E088000D70A0319D80ADC0A102B5908FB
:1006B800303EDE00831358188317570884005E08FD
:1006C8008000D70A0319D80A8313581883175708C4
:1006D8008400800156088A00550882008313831617
:1006E800031358188317570884000008003A8A1122
:1006F8000A12031D802B842BD70A0319D80A722BE0
:1007080003110319882B892BAD2B8E2B5A088A00CD
:10071800590882008A2383160313DB0083135818B1
:100728008317570884005B088000831358188317C1
:10073800570884000008003A8A110A120319A52BE9
:10074800A62BAD2BD70A0319D80AD90A0319DA0A36
:10075800842B56088A005508820004306A02031C5C
:10076800B92B031DB92B003069020318BC2BCB2B06
:1007780001308312E1000030E0000000E00BC12BE3
:10078800000000308316E902031CEA03B12B003095
:100798006A02031CD32B031DD32B043069020318F0
:1007A800D62BE72B6A088312E100831669088312A7
:1007B800E0000310E10CE00C0310E10CE00C000079
:1007C800E00BE32B0000080063086404031DED2B15
:1007D800FB2B8312E101FA30E0000000E00BF12B63
:1007E800000001308316E302031CE403E82B080031
:1007F800831205158316690EF039831286040F38A3
:100808008605051108008312851183166308E9001F
:10081800E90E0F30E905FC2383166308E900FC2381
:100828008316EA012830E900B12308008312031374
:10083800851583166308E900E90E0F30E9058A116A
:100848000A12FC2383166308E900FC238316EA01D5
:100858003230E900B123080083160313061286120A
:100868000613861385110511E4010F30E300E82310
:100878008312851103308316E900FC238316E401F3
:100888000530E300E8230330E900FC238316EA017E
:100898006430E900B12303308316E900FC23831692
:1008A800E4010530E300E8230230E900FC23831665
:1008B800EA012830E900B12328308316E300072431
:1008C80008308316E30007240F308316E30007245B
:1008D80001308316E30007248316E4010230E300A5
:1008E800E8230630E30007248312031721088A004F
:1008F80020088200A9010130AA000230AB000330B1
:10090800AC00031334030317A3002308003C031CA3
:100918008E2CE42CA20123082202031C942CE12C27
:100928000130AE00293022070318AE0A83132E18AF
:10093800831784000008A6000130AE002A30220781
:100948000318AE0A83132E18831784000008A70023
:10095800AE013B3027070318AE0A83132E188317FE
:1009680084000008AD00B2013B3026070318B20A24
:1009780083133218831784000008B10031082D0250
:10098800031CC72CDF2C0130AE00293022070318C6
:10099800AE0A83132E1883178400270880000130BD
:1009A800AE002A3022070318AE0A83132E188317C5
:1009B800840026088000A20A8F2C0130A302892C0B
:1009C8000308A8007F308305A401A201031334089B
:1009D80003172202031CF12C4C2D0130AE002930E4
:1009E80022070318AE0A83132E1883178400000801
:1009F800A600AE013B3026070318AE0A83132E1853
:100A0800831784000008AD002408AD02B2013F300E
:100A180022070318B20A83133218831784002D089B
:100A28008000AE013F3022070318AE0A83132E1848
:100A3800831784000008A4070130A500B2013730ED
:100A480026070318B20A8313321883178400000894
:100A58000739F83E031C322DA5013A2D0739031931
:100A68003A2D0310A50DFF3E031D352DAE012508B7
:100A7800FF3AAE09AD00B201433022070318B20AAB
:100A880083133218831784002D088000A20AEA2CE9
:100A9800A6010130A2000313340803172202031C25
:100AA800562DAF2DAE013F3022070318AE0A83132F
:100AB8002E18831784000008003A0319642D7B2D33
:100AC800AE01433022070318AE0A83132E1883178A
:100AD80084000008AD00B201433026070318B20AAB
:100AE80083133218831784002D088005AD2DA60ABC
:100AF80026082206031D812DAD2DAE013F302207A9
:100B08000318AE0A83132E18831784000008AD005B
:100B1800B2013F3026070318B20A8313321883172D
:100B280084002D088000AE01433022070318AE0A66
:100B380083132E18831784000008AD00B2014330D8
:100B480026070318B20A83133218831784002D0866
:100B58008000A20A4F2D260A0313B5003508031793
:100B6800A20004302202031CBA2DD12DAE013F3061
:100B780022070318AE0A83132E18831784008001F6
:100B8800AE01433022070318AE0A83132E188317C9
:100B98008400FF308000A20AB52D0130A200043085
:100BA8002202031CD82DF32DAE013F302207031873
:100BB800AE0A83132E18831784000008003A031D19
:100BC800E62DF12DAE013F3022070318AE0A83133C
:100BD8002E188317840001308002A20AD32D28081A
:100BE800830021088A002008820004305702031C71
:100BF800FE2D4D2E0130D80057080739F83E031C4A
:100C0800072ED8010F2E073903190F2E0310D80D00
:100C1800FF3E031D0A2E58088312B6048316DC0112
:100C28005808FF3ADC09831286058316DA018630F4
:100C3800D900DC015808FF3ADC09DB0083135A1895
:100C48008317590884005B088005DC01373083125C
:100C5800340783160318DC0A831383165C1883177A
:100C6800840057088000DC013B3083123407831668
:100C78000318DC0A831383165C18831784007F30FB
:100C880080008312B40A06300317A1004D30A0007B
:100C98007E2C8316031356088A0055088200831297
:100CA8000313B601B501B4018316D7010630D60087
:100CB8006130D5008A110A12F92D0130D7000630AB
:100CC800D6006830D500F92D0230D7000630D6009E
:100CD8006F30D500F92D0330D7000630D6007630B6
:100CE800D500F92D7F308312C700C80106300317DD
:100CF800A1008030A000302C0C3083160313E300D1
:100D080007248316C201C301031103198C2E8D2EEB
:100D1800832F831247088316C0008312480883165E
:100D2800C1008312E001E1015F0884008407683094
:100D380084078313840A8017840360088000840A68
:100D480061088000AB30E00006305D286928831216
:100D580003135F0884008407683084078313840AB8
:100D68008A110A12801FAA2E831641088312480688
:100D7800031DBF2E022F831641080139C900C90D72
:100D8800C90DC90DF830C90541080239CD00031055
:100D9800CD0C4D080139E300E30EE30DE30DC0303F
:100DA800E3058030E30449083F39E3040724203091
:100DB8008316E3001A248312480801398316C900F0
:100DC800C90DC90DC90DF830C90583124808023983
:100DD8008316CD000310CD0C4D080139E300E30E56
:100DE800E30DE30DC030E3058030E30449083F39E3
:100DF800E30407242A308316E3001A2483164008E4
:100E080083124706031D092F7E2F04304802031C56
:100E18000E2F242F8316C6013B30831248078316F2
:100E28000318C60A8313831646188317840083128F
:100E38004708800007300317A1002430A0007E2C4B
:100E480083160313D801B630D700831247088316D8
:100E5800D9000730D6003230D5000E2BD801B63075
:100E6800D7000730DA00C730D9000730D6003E3047
:100E7800D500722B8312480801398316C900C90DA1
:100E8800C90DC90DF830C9050130C90783124808D2
:100E980002398316CD000310CD0C4D080139E3004B
:100EA800E30EE30DE30DC030E3058030E3044908A9
:100EB8003F39E30407248316CA01B630C9008313F7
:100EC8004A188317490884000008D5005508003AD5
:100ED800031D6F2F7E2F5508E3001A248316C90AB5
:100EE8000319CA0A83134A1883174908840000089B
:100EF800D5006A2F8316C20A0319C30A882E35083B
:100F08008A0034088200643400340A34003410340F
:100F18002734E8340334643400340A3400340034A9
:100F2800CA349A343B340034E134F534053480341F
:100F3800963498340034403442340F340034A034AA
:100F48008634013400341034273400340034E83453
:100F580003340034003464340034003400340A3478
:100F680000340034003430343134323433343434DF
:100F780035343634373438343934413442344334F0
:0A0F8800443445344634203400346C
:02400E00103F61
:00000001FF
